:10000000F01F001055380000513800005138000032
:100010005138000051380000513800000000000045
:100020000000000000000000000000005138000047
:100030005138000000000000513800001116000087
:10004000E1130000E1130000E1130000E1130000E0
:10005000E1130000E1130000E1130000E1130000D0
:10006000E1130000E1130000E1130000E1130000C0
:10007000E11300004D3800004D3800004D380000FD
:10008000C9160000E1160000F91600001117000063
:100090004D380000D91700004D3800004D380000E1
:1000A0004D3800004D3800004D3800004D3800003C
:1000B0004D3800004D3800004D3800004D3800002C
:1000C00008B500230B60036000F00CFE08BD08B506
:1000D0000A20002101F098FA08BD000038B5094B4C
:1000E0000D1C041C1968012001F03EFB012001F0E9
:1000F0001BFB291C201C02F00DFF012001F024FB3A
:1001000038BDC046B004001070B5054E051C0E2465
:10011000013C295D301C01F081FD002CF8D170BD3F
:10012000843A000038B5164801F078FD154C201CC3
:10013000FFF7EAFF144D4221281C01F06FFD201C3F
:100140000E30FFF7E1FF4321281C01F067FD201C62
:100150001C30FFF7D9FF0D4801F060FD201C2A304C
:10016000FFF7D2FF281C4E2101F058FD201C38302B
:10017000FFF7CAFF616D064801F050FD38BDC0466B
:10018000873A0000B80400108D3A0000943A00004D
:100190009A3A000008B5074B0120196801F0E4FA0B
:1001A000012001F0C1FA02F04DFE012001F0CCFA6D
:1001B00008BDC046B004001010B5041C0D2107484E
:1001C0000C2200F09BFC00F0FBFB201C0021032212
:1001D00000F00AFD00F0FEFB10BDC0461F3C000011
:1001E00013B59620000201F035FB1248FFF7E4FF3B
:1001F000FFF7D0FF1048114901F010FD002401F075
:10020000CFFB002802D001F005F800240A2001F0FD
:100210002BFA684601A9FFF753FF009B002B03D17F
:10022000074B01349C42EADDFFF7B4FF054801F0BB
:10023000F5FC13BDA63A0000B53A0000C03A000034
:100240006F170000C73A000000B5074B89B01A7855
:10025000064B68461B78064901F0EBFC6846FFF741
:10026000ABFF09B000BDC046B8010010000000108F
:10027000D23A000013B5FFF7E7FFFFF78BFF00242A
:10028000684601A9FFF71CFF009B002B2CD0182B00
:1002900021D004DC142B0DD0152B20D104E0342BFD
:1002A00012D0352B1BD107E0134B00241A783E2ABD
:1002B00016D806E0104B08E0104B00241A78062AE6
:1002C0000ED801321A700BE00C4B1C78002C07D0B2
:1002D000013C1C7003E0FFF75DFF282400E00024D0
:1002E00000F05AFBFFF7B0FFC820013401F0BCF961
:1002F0001D2CC5DD13BDC046B80100100000001064
:1003000073B5124B041C1249186803F025FB114900
:100310000090114A114B201C01F08BFC00F0C4FD31
:10032000002812D000F0DCFDFA218900051C03F042
:1003300013FB061C201C01F0C9FC094B2018734359
:100340000849EB18321C01F074FC73BDB4040010B2
:1003500040420F00E03A0000C03A0000ED3A0000D1
:1003600018FCFFFFF03A000070B50D1C161C041CB1
:1003700000F026FB0B480D210C2200F0BFFB281CCF
:10038000A1B2002200F030FC07480321062200F051
:10039000B5FB301C0121092200F026FC00F01AFBFD
:1003A00070BDC0461F3C00005C3B000010B588B02B
:1003B000041C6846FFF7A4FF69466A46201CFFF745
:1003C000D3FF08B010BD000073B518200021FFF75F
:1003D00085FE424E0024424D983600E0404D0120FB
:1003E00001F0B2F9002C01D0002000E0062001212C
:1003F00001F00AF9684601A9FFF762FE009B002B95
:1004000021D1002CF0D13368002B0DD0354B009456
:100410001A6811321A6004E002F0BEFC009B01333E
:100420000093009B102BF7DD2F4BED18DED5182025
:100430000021FFF753FE294B94331C6863425C4153
:1004400000F072FACEE7002C03D0182BC7D100F0D1
:10045000C9FA009B182B2BD1019B00220192822B01
:1004600022D004DC322B0ED0732B20D119E0832B49
:100470000FD0C22B1BD11D4B196801311960022905
:1004800016D11A6014E01A4B01201B68C01A00F044
:1004900039FD0120FFF78AFFFFF77CFEFFF717FE0B
:1004A00006E0FFF79DFE03E0FFF7E4FE00E00193A6
:1004B000104B0120196801F057F9012001F034F9BF
:1004C0000098019902F026FD044B002494331B6828
:1004D000002B83D100F028FA01247FE7B804001034
:1004E00020BF0200E40200100CFEFFFF900100108C
:1004F00008000010B004001013B501F017FC00F064
:10050000BDFB00F06FFA1C48002100F01DFF002128
:100510001A4800F019FF00F057FC002004210122C6
:1005200000F0A0FE0020021C042100F0E9FE0020E3
:100530000521012200F096FE00200521021C00F09A
:10054000DFFE00F073FE3C24201CFFF72FFF013C70
:100550001E2001F089F8022CF6D102F03FFB1E2389
:1005600000930B230193064806490022064B02F034
:10057000EFFBFFF729FFC046984004409C40044031
:1005800009380000C1000000E402001000B500E0DE
:1005900001300378202BFBD000BD00B5031C303B9D
:1005A000DAB2092A01D8181C08E020231843031CDA
:1005B000613B5738052B01D90120404200BD70B581
:1005C0000E1CFFF7E3FF0025041C06E0FFF7E5FF24
:1005D000002805DB2D010543013420780028F5D1E2
:1005E0003560201C70BD000008B500F079FC011CCE
:1005F000014801F013FB08BDFB3A000000B5C30041
:10060000181A064BC0180723013BC25C002A03D10D
:10061000002BF9D1012000E0002000BD540500109E
:100620007FB5194801F0FAFA00250326354219D1A1
:10063000281CFFF7E3FF002810D0681CFFF7DEFF3F
:1006400000280BD0A81CFFF7D9FF002806D0E81C13
:10065000FFF7D4FF002801D004350FE00B48291C18
:1006600001F0DCFA291C684601F0CAFB6846FFF776
:100670004BFD074801F0D2FA6C1C251CFF2DD5DD7F
:10068000FFF750FD7FBDC046C03A0000073B0000A9
:10069000D35F000070B50E1CFFF778FF0D25041C1A
:1006A0002078FFF77AFF002807DB01347055013D01
:1006B000F6D2201CFFF76AFF00E0002070BD0000AA
:1006C00030B5464C87B023680868002B06D14448F3
:1006D00001F0A4FA02F082FA012357E0012B12D1B3
:1006E0008379202B07D0002B05D03E49062201F04C
:1006F00000FB002803D1394B1A6801326AE03A48FE
:1007000001F08CFA5EE00378412B1BD1374C0230AC
:10071000211CFFF7BFFF002854D00378422B51D192
:10072000211C02300E31FFF7B5FF00284AD00378B4
:10073000432B47D1211C02301C31FFF7ABFF0028AF
:1007400049D13FE04D2B23D1294D0230291CFFF721
:10075000A1FF002836D003784E2B33D1291C02305C
:100760000E31FFF797FF00282CD00378472B29D1B3
:10077000023005A9FFF723FF059B002B22DB2A3D52
:100780006B651C481C4901F049FA0023236022E0F4
:1007900005A9FFF714FF0378041C202B01D0002BC0
:1007A00010D10025201C01A9FFF774FF0599041C36
:1007B000691801A801F038FB002C03D00135042D85
:1007C000F0D108E002F00AFA0A480C4901F026FAD2
:1007D000024B00221A6007B030BDC046BC020010B8
:1007E000103B0000C03A0000263B0000B804001097
:1007F000E2040010323B00003C3B00003F3B0000A5
:1008000037B54C6824E0201CFFF7C0FE01A9FFF7B4
:10081000D6FE019B041C002B1DD0D8B2FF2B09DD96
:1008200000F0FCF9051C01980012C0B200F0F6F9C6
:10083000019003E000F0F2F90025019001980028F2
:1008400002D0291CFFF74AFC23785A1E9341E41872
:100850002378002BD7D137BD08B5064A012113787C
:100860004B40137001D0044900E00449044801F0F2
:10087000D5F908BD9D030010463B0000493B000030
:100880004D3B000070B5051C01200821021C00F042
:1008900037FD0724012601200821002200F030FD49
:1008A0002A1C224132400020022100F029FD0120B3
:1008B0000821021C00F024FD013CECD270BD10B5F3
:1008C0000021041C0A1C022000F01AFD201CFFF766
:1008D000D9FF10BDF7B5012300930023019372B631
:1008E0006C46061C02AF01CC50235B421843C0B2D9
:1008F000FFF7E5FF0020FFF7E2FF1020FFF7DFFF23
:10090000E020FFF7DCFF002502200021012200F09B
:10091000F7FC705D0135FFF7B5FF842DF4D1843607
:10092000BC42E0D162B6F7BD08B5AC20FFF7C7FF07
:10093000AE20FFF7C4FFA520FFF7C1FF08BD38B503
:100940000D1C041C012200F08DFC291C201C01221E
:1009500000F0D6FC38BD08B5AF20FFF7B0FFA420EB
:10096000FFF7ADFF08BD08B5AE20FFF7A8FF08BD33
:1009700010B5041CF820FFF7A2FF201CFFF79FFF13
:1009800010BD10B5041C8120FFF799FF3F202040C7
:10099000FFF795FF10BD000008B5074B20201B781E
:1009A0001843FFF78CFF0A2000F05EFE034B187817
:1009B000FFF7E7FF08BDC04600000010B8010010B7
:1009C00008B5842202480021520001F05FF908BDF9
:1009D000A503001008B50248FFF77CFF08BDC0461C
:1009E000A503001008B501200821FFF7A8FF00208B
:1009F0000221FFF7A4FF02200021FFF7A0FF022041
:100A00000621FFF79CFF0320011CFFF798FF03203E
:100A1000011C002200F074FC02200621002200F0DC
:100A20006FFC06210122022000F06AFCFFF7C8FFDC
:100A3000FFF7D0FFA220FFF742FFA020FFF73FFF04
:100A4000C020FFF73CFF0020FFF792FF0A2000F0D4
:100A50000BFE4020FFF733FF2C20FFF730FF322042
:100A600000F002FE2E20FFF72AFF322000F0FCFDEE
:100A70002F20FFF724FF0A2000F0F6FDFFF78CFF80
:100A8000AF20FFF71CFFA420FFF719FF08BD0000EF
:100A900000B50F290ED883280CD8CB0884225343E5
:100AA0000722C0181140044B80220A41111C1A5C15
:100AB0001143195400BDC046A5030010F0B55B18E2
:100AC000DBB216E08425CC086C4307270F40802555
:100AD00004193D41EFB2A6189C4605E0064BE51807
:100AE0002B7801343B432B70B442F7DB0131634672
:100AF000C9B29942E6D3F0BDA503001000B5074B7B
:100B00001860074B1970074BD1081A70064B197003
:100B1000500701D00131197000BDC046A00300107C
:100B2000AD040010AE040010A4030010F0B589B0AD
:100B3000059106925A2800D92020284B284A1B6884
:100B400093420BD1440003212418623C019103918C
:100B50000EE0195D01320231641802E00024221C0B
:100B600020388242F5D31A5D1B195B7801920393FA
:100B700000252CE06B430199FA188A4215D2174AD6
:100B800000261268D2191219D3189B7804930123F6
:100B9000049AB340134205D0029B07989919C9B231
:100BA000FFF776FF0136082EF1D1029B013708339B
:100BB000DBB2029306E0059A06995319DBB2029163
:100BC0000027079307490B789F42D3D30135039A37
:100BD0009542F0D109B0A8B2F0BDC046A003001004
:100BE0005C3B0000A4030010F7B5061C0C1C01922E
:100BF00001F06CF800250090832708E06B46705DDB
:100C0000E1B21A79FFF792FF013024180135A742AB
:100C100002D3009B9D42F1D3F7BD000000B50F2326
:100C2000020918408000031F00D52833002B0EDB7B
:100C3000511E0320884280414042002807D1242BC6
:100C400006DC04218A1A0349CB18985C00E00020D6
:100C500000BDC0462240000070B5064E051C0024B1
:100C6000A05D054B291CC018013400F06DFB0A2C57
:100C7000F6D170BD5E40000000400440F8B5102081
:100C8000FFF7EAFF094C271C143725786678281CE3
:100C9000311C002200F0E6FA0234281C311C01222B
:100CA00000F02EFBBC42F0D1F8BDC0464A40000027
:100CB000F8B50B4C271C143725786678281C311C96
:100CC000012200F0CFFA0234281C311C002200F06F
:100CD00017FBBC42F0D10020FFF7BEFFF8BDC046B5
:100CE0004A400000F0B589B0002404900591FFF758
:100CF000C5FF0220072101220694079400F0B2FAF2
:100D000002200721221C00F0FBFA201C0B2100F01E
:100D1000CDFAA04202D11823069301240021264DCA
:100D200003916A782F78111C0192381C012200F07F
:100D300099FA381C0199002200F0E2FA03231F4EB1
:100D4000029314E03078717800F0B0FA002807D1EF
:100D500003991B4AA3008A5C183369465A50013430
:100D6000029A039B013A013302920393023EE30F7E
:100D700000210122A2424B41DBB28B4202D0029BF6
:100D80008B42DFDA381C0199002200F06BFA0199DE
:100D9000381C012200F0B4FA0A4902358D42C0D154
:100DA000201E06D0069B049A05991360079B01201C
:100DB0000B6009B0F0BDC0464A4000002040000072
:100DC000224000005E40000008B50120021C0B21FB
:100DD00000F048FA01200B21002200F091FA0320D4
:100DE0000221012200F03EFA03200221002200F03D
:100DF00087FA08BD37B5234B10211A68051C8A43B2
:100E00001A60214B8022196892010A431A6001205E
:100E10000B21002200F026FA01200B21002200F015
:100E20006FFA1A4B9F211A68194C8A431A601A6884
:100E300018491A60184B186802F08EFD80230002D2
:100E400018432A1C20600221032000F059FA1420C4
:100E500000F00AFC2368FF229343236023680F4AB3
:100E6000134323600E4B1A680192019A002AFADAA2
:100E700022680C4B13402360FFF7A6FF0198000483
:100E8000800D3EBD3882044080800440984004407C
:100E900000C0014000093D00B404001080000001C2
:100EA0002CC00140FFFFFFF810B50C4C2068002853
:100EB00013DA00202060FFF79DFF0A280ADC0120DA
:100EC000FFF798FF0138C023FF385B00984201D834
:100ED00001232360FFF778FF206810BD0400001095
:100EE00008B5FFF7E1FF011E08D00120FFF782FFE0
:100EF000011E03D0024802F02FFD011C081C08BD92
:100F000050BB120010B500280DD0254B80211A6867
:100F10008A431A60234A012311681942FCD0224BEC
:100F200003221A6001E0204B1860204B01220021AF
:100F30001A6019601A6019681142FCD01C4B01221A
:100F40001A601C4A802114684902214311601A1C4E
:100F5000002804D1124B8024196821431960164BD4
:100F6000196888421AD01860002801D0134800E0A0
:100F70001348116802F0A2FC124C2121206002F0FB
:100F8000EBFC114B18609620000200F063FCFA2184
:100F90002068890002F0E0FC00F04CFB10BDC04668
:100FA000388204400C800440708004407480044007
:100FB000788004408080044008000010006CDC024F
:100FC000001BB700B4040010B004001008B500F016
:100FD0003BF9134B00211A68120B12031A60114BD4
:100FE0001A68120B12031A600F4B1A68120B1203C5
:100FF0001A600E4B1A68120B12031A600C4B012276
:1010000019600C4B1A6019601A6019681142FCD003
:10101000094B23221A600120FFF774FF08BDC04668
:10102000008000500080015000800250008003507A
:1010300040800440448004400880044070B50F495B
:101040000F4800F0EBFD0F4800F0E8FD0E4E0F4D8D
:1010500000242B196159DA68301C0A4B143400F053
:10106000DDFD782CF5D10A4800F0D8FD00F018FB22
:10107000011C084800F0D2FD70BDC046C03A000017
:1010800068400000B9400000794000000C000010EA
:1010900084400000A6400000F0B53C4B8BB01D68BA
:1010A000002D3AD03A4B02901B6801209B685DE00E
:1010B00001342378202BFBD0002B3AD0B300083327
:1010C0006A469C500136FF2D01D135E0013423786A
:1010D000202B01D0002BF9D1202B02D1002323702B
:1010E0000134012E1BD12A4F2A4B07223B6001926B
:1010F0003D1C09E02B680298196800F009FE0028E1
:1011000008D02B6814332B60019B013B0193002B0B
:10111000F0D132E03B681D7901E0041C2E1C2378DD
:10112000002B06D000230722B2425B41DBB2002B2A
:10113000BFD1002E1CD000E00025154C022E05D199
:101140000398154900F0E4FD002801D0AE420AD80A
:1011500023681248D96800F061FD236810481969B6
:1011600000F05CFD04E02368F0B29B6802A9984798
:10117000064B1B68002B07D103E00198011CFFF709
:101180005DFF084800F04AFD0BB0F0BDBC02001046
:10119000C40200100C000010B3400000B540000075
:1011A000373B0000BC40000038B5041C154D0A2830
:1011B00008D002D808281CD110E00D2802D07F28C2
:1011C00017D10BE02B6800221A700F4800F026FDA3
:1011D0000E4C201CFFF760FF2C6012E02A680B4BBE
:1011E0009A420ED90A48211C00F018FD2B68013BD9
:1011F00006E00748211C00F011FD2B681C7001332C
:101200002B6038BDC0020010B9400000B9010010C9
:10121000C840000008B503E000F0A0FBFFF7C4FFE2
:1012200000F0BEFB0028F7D108BD000008B5034A56
:10123000034B04481A6000F0F1FC08BDB90100102E
:10124000C0020010BC400000044B40211A680A4351
:101250001A60034B01221A707047C0468080044018
:10126000C802001070B50E4B061C1B780D1C141C18
:10127000002B01D1FFF7E8FF013E022E03D8094BF6
:10128000B600F35800E0084B1A68012C03D1AC40BB
:1012900014431C6003E00124AC40A2431A6070BDFB
:1012A000C80200104C4100000080005038B50F4BC0
:1012B000051C1B780C1C002B01D1FFF7C5FF00207B
:1012C000032D11D8281C012302F0E4FA02040608B9
:1012D000074A04E0074A02E0074A00E0074A1068AC
:1012E000A3401840431E984138BDC046C8020010B4
:1012F000FC3F0050FC3F0150FC3F0250FC3F0350BC
:1013000070B50E4B061C1B780D1C141C002B01D154
:10131000FFF79AFF013E022E03D8094BB600F3589F
:1013200000E0084B1A68012C03D1AC4014431C6048
:1013300003E00124AC40A2431A6070BDC802001053
:1013400058410000FC3F005038B5084B041C1B7886
:101350000D1C002B01D1FFF777FF23681822934360
:10136000236023681D43256038BDC046C8020010B5
:101370001F234209184001238340181C014B92008F
:10138000D050704700E100E01F23420918400123BC
:101390008340181C2032024B9200D0507047C04648
:1013A00000E100E0054B3F221A60054B01221A6064
:1013B000044B40211A688A431A6070472480044015
:1013C000D88004403882044008B5044B40211A6894
:1013D0008A431A60FFF7E6FF08BDC0463882044022
:1013E00008B5154B1868FFF78DFD0720FFF7CCFFF8
:1013F0000820FFF7C9FF0A20FFF7C6FF0C20FFF700
:10140000C3FF0B20FFF7C0FF0920FFF7BDFF0B4A0A
:101410000023136001210A4A49421160094A1360FE
:10142000094A1360094B01221A60094B1A680132FC
:101430001A60C04608BDC04608000010048204407F
:101440000882044004C000403CC0004000C000408E
:10145000CC02001008B5FFF72BFC0A480021FFF76B
:1014600073FF09480021FFF76FFF08480021FFF7CD
:101470006BFF07480021FFF767FF06480021FFF7D1
:1014800063FF08BD0840044000400440AC400440F5
:10149000144004401C400440F8B5071C0C1C72B6F4
:1014A000FFF7D8FF434B1A68434B1A60002F01D057
:1014B000424B00E0424B434A04211360424B434DF0
:1014C0001A680A431A6000232B609C4218D0072038
:1014D000FFF74EFF0820FFF74BFF0A20FFF748FFFA
:1014E0000C20FFF745FF0B20FFF742FF384B394A2E
:1014F00019680A401A602A68EC235B0113432B60C9
:10150000002F4FD0344B354C354900260E60201C3F
:101510001E60311CFFF718FF301C0921321CFFF739
:10152000A1FE301C0921321CFFF7EAFE2D4B802260
:10153000196811431960236807218B4323602368CE
:1015400002210B4323607B00DB1999015B189B0090
:101550002549DF19254B0F6003211960244B2549CC
:10156000186801401960196809200A431A60FFF7DA
:10157000FFFE174A802311689B00194311602A68F7
:10158000022113431C4A2B60012313601B4A116084
:101590001B4A134913601660136010681842FCD090
:1015A00001230B60174B012252421A6062B630BF12
:1015B000F8BDC0463882044034820440BF180000A1
:1015C000FF1800003082044010ED00E00482044067
:1015D000008204407FE2FFFF044001406440044079
:1015E00004C000408080044018C0004014C0004087
:1015F0003CC000400FF0FFFF788004407080044042
:10160000748004400882044008B5FFF745FF08BD18
:1016100000B5064B1A6801321A601B68013303D10A
:10162000034B1A6801321A6000BDC046D402001094
:10163000D002001000B5074B98420AD8064A002392
:101640001360064A01381060054A1360054B0722F3
:101650001A6000BDFFFFFF00D402001014E000E09C
:1016600018E000E010E000E000B50C4A1368002824
:1016700000D10120C1438B4204D809E011688142A6
:10168000FCD301E0591C081811689942F6D203E016
:101690001168C91A8142FBD300BDC046D4020010B4
:1016A00010B5064BFA211868054B89001C6802F03A
:1016B00005F9044B5C43201810BDC046D40200104D
:1016C000D002001037894100034B01221A60034BFE
:1016D0001A6801321A60704700C00040D80200103A
:1016E000034B01221A60034B1A6801321A607047DB
:1016F00000000140DC020010034B01221A60034B82
:101700001A6801321A60704700400140E002001080
:10171000034B01221A60034B1A6801321A607047AA
:1017200000800140E402001000B5002803D1044B02
:1017300001221A6003E0012801D1024B186000BDAC
:10174000044001400480014000B5002802D1044B50
:10175000186004E0012802D1024B00221A6000BD8B
:10176000044001400480014010B500280FD1124B05
:1017700080221C68920022431A60104B03221860DA
:101780000F4B19600F4B1A608022D20211E0012822
:1017900011D1094B80221868D20002431A600A4B0B
:1017A00000221A60094B03221960094B1A6080223B
:1017B0001203084B1A6010BD80800440E002001044
:1017C0001840014014400140E4020010188001401C
:1017D0001480014000E100E008B5184B1A680E23A0
:1017E0001340062B0DD1164B9E221B68DBB2134211
:1017F00004D0144A5360144B1B681EE0D9071CD553
:1018000001E0042B05D1104B1868C0B200F0B7F806
:1018100013E00C2B06D10B4B8022596852000A436F
:101820005A600AE0022B08D1054B1A68054B910655
:1018300001D5002200E001229A6008BD0880004026
:1018400014800040E802001000800040004870470B
:10185000E802001070B52A4C2A4B80229203DA6706
:1018600000219022061C201C00F010FA0023A36027
:1018700000F06EF8244B07251A68244CAA431A601E
:101880001968012211431960214B1968A943196095
:101890001968114319601F4B8021186849010143E1
:1018A00019601D4B1A608322226019681B4B18684F
:1018B00002F004F8311C000902F000F81849030A8C
:1018C000184A0B60C0B2032310602360164B1D60E2
:1018D000164B186860201C680440602CFBD101E0A6
:1018E000146800E001201C680442F9D1044B012275
:1018F0001A700F4B802292031A6005230B6070BD93
:10190000E802001004E100E0A44004400C80004024
:10191000A84004408080044098800440B404001033
:101920000480004000800040088000401480004097
:1019300000E100E000B5044A202311681942FCD000
:10194000024B186000BDC04614800040008000407B
:1019500008B5FFF77BFF0023437308BD08B5FFF709
:1019600075FFC27B031C8218107CDA7B7F21013259
:101970000A40DA735A7B013AD2B25A7308BD10B5E5
:10198000041CFFF763FF837B7F22C3181C74837BD7
:10199000013313408373437B0133DBB2437310BDC8
:1019A00008B5FFF753FF407B431E984108BD30B593
:1019B000002402E00570013401301D5D002DF9D1D5
:1019C000121B131C02E00170013B0130002BFADCFA
:1019D000D043C0170240A01830BDF8B5051C0F1C3D
:1019E0001E1C541E092B01D800240FE0181C0A21CC
:1019F00001F064FF221C031C391C281CFFF7EDFFBB
:101A0000041C2D1805E02F7001340135013A002A1D
:101A1000F9DC301C0A2101F095FF30312970601C7F
:101A2000F8BDF8B50C1CD9175F18061C4F40551EA1
:101A3000092F12D9381C0A21002B03DA01F03EFFCE
:101A4000434202E001F03AFF031C211C2A1C301C17
:101A5000FFF7E7FF041C351813E0002B00DA951E92
:101A6000002201E0B4540132A91A0029FADCEC4347
:101A7000E4172C403519002B03DA2D232B70013489
:101A80000135381C0A2101F05DFF30312970601CDE
:101A9000F8BD73B5069E041C1D1C3009531E00289A
:101AA0000AD000901A1C201C2B1CFFF7F2FF2418F0
:101AB00005E0217001300134013A002AF9DC0F23DE
:101AC0001E40092E01D8303604E0002D01D03736F3
:101AD00000E057362670013076BDF0B585B0041CA5
:101AE0000F1C002801D00021017000256BE0252982
:101AF00003D021700132013405E05178252904D149
:101B000021700232013401355DE0302903D0013209
:101B10000292202101E002320292029E9C4632781B
:101B20002D3A50424241B6180296002205E00A239F
:101B30005A438218303AD2B201363078031C303B17
:101B4000092BF4D90296AE186346BE4201D97A1B1E
:101B5000D2B269280ED006D863282CD0642809D0C8
:101B600058283ED119E075280AD078280FD073285C
:101B700037D11AE01E1D201C1B68FFF752FF04E03E
:101B80001E1D201C1B68FFF728FF331C17E01E1DBD
:101B90001B68201C0093002304E01E1D1B68201CF2
:101BA00000930123FFF775FFEFE71E1D201C1B6844
:101BB000FFF7FDFEE9E71A68012022700433029A5C
:101BC000241801322D181178BD4201D200298ED17E
:101BD0000023BD4201D2237005E0013C2370013D8A
:101BE00001E001256D4205B0281CF0BD10B50C1CAC
:101BF000131C6421221CFFF770FF10BD00B5031CED
:101C00009BB00A1C01A8191CFFF7F0FF632800DD38
:101C1000FEE701A800F0A6F81BB000BD0FB407B5A1
:101C200004A901C90191FFF7E9FF03B008BC04B0A2
:101C300018470EB403B503AA02CA0192FFF7D6FFF4
:101C400002B008BC03B0184770B50323041C184247
:101C500005D10D1C041C194201D1934201D300236C
:101C600011E0131C40CD043B40C4032BFAD8141FD1
:101C7000A4080134A400032309191A400419EEE74B
:101C8000CD5CE55401339342FAD170BD30B50B04FD
:101C90000D061D430D430B021D430323041C9342F9
:101CA0000DD218420BD1131C043B20C4032BFBD8CC
:101CB000141FA4080134A40003231A4004190023AC
:101CC00001E0E15401339342FBD130BD00B5002364
:101CD00000E00133C25C002AFBD1181C00BD00B536
:101CE000031C01E0013101330A781A70002AF9D18E
:101CF00000BD30B5031C002406E01D5D085D281AF8
:101D000005D10134002D02D09442F6D1002030BD1F
:101D100000B502E00130002B06D00A7803780131CB
:101D20009342F7D0981A00E0181C00BD08B5FFF7E1
:101D30004DF90B4BFA211868890001F00DFEFFF7F1
:101D400079FCFFF781FAFFF73FFB96200002FFF7CF
:101D500081FDFEF747FEFEF733FEFFF767FA08BD89
:101D6000B404001010B5041C02E00134FFF7E2FDDA
:101D700020780028F9D110BD30B5F8238A01DB00A6
:101D800013404A05920E1343F822120211401943E0
:101D90000A235943CA1083181C1CEB345D7824783D
:101DA000EA336C401B7824021C43835C201C58409F
:101DB0000723194008418005800D30BD08B5054B4B
:101DC000011C984201DD044BC1180448EA38FFF7B2
:101DD000D3FF08BDFF17000000F8FFFF64410000BB
:101DE00008B54018511A013101F018FE08BD08B5B8
:101DF000801889189A1A0132FFF726FF08BD0000E3
:101E000010B5CB00591A074B0F22C9180023CC5C20
:101E100014400470CC5C0133240944700230072B59
:101E2000F5D110BD5405001010B5CB00591A064B62
:101E3000C91800234278047812012243CA5401339E
:101E40000230072BF6D110BD5405001030B5B14B50
:101E500087B0D96EB04D4A1E91416A46D175A96AC4
:101E60001A1CC806400F0138062807D801F012FDD9
:101E7000040C1F1217191C00022409E05A6E1632B6
:101E80009200D3581C1C15E05B6E16339B00D4588F
:101E900000230FE09B6DD46DA3420ADC0AE002240C
:101EA00003E00C24032305E00D24231C02E00D2491
:101EB000EEE70D242C6148111F2800D922E16A4663
:101EC0001732944901F0F0FC2000220028002A007B
:101ED0002D002F00380040004400490051005F00F1
:101EE00067006F00770085009300A200B400C30074
:101EF000D500D300E300E600E900F100010105018F
:101F00000F01110113011901081C00E08348191C7D
:101F1000221CFFF765FFF5E08148F8E70A1C0E3246
:101F200003E07E4809E00A1C1C32081C111C1A1C24
:101F3000231C01F0F9F8E5E07948011C0E391A1C60
:101F4000231CFFF754FFDDE07448011C0E31EEE75F
:101F50000A1C1C32081C111CF1E70A6E1020002A12
:101F600000D00A200A1C0E3206E00A6E1020002A59
:101F700000D00A200A1C1C3200946C4617340290D0
:101F80000194081C51E001201070086E10220028F6
:101F900044D00A2242E00A6E1020002A00D00A2013
:101FA0000A1C0E320EE001201070086E102200286C
:101FB00055D00A2253E00A6E1020002A00D00A20D1
:101FC0000A1C1C3200946C46173402900194081CC1
:101FD00078E00A6E1021002A00D00A21504A684693
:101FE0001730019002910094101C111C1DE00A6E24
:101FF0001020002A00D00A20494A00946C46111C87
:10200000173402901C390194101C0EE0096E012057
:1020100010701022002900D00A224149684617306A
:10202000019002920094081C002201F087F869E0F8
:102030000A6E1020002A00D00A20394A00946C460B
:10204000111C173402901C390194101C3AE0096EDF
:10205000012010701022002900D00A223049684661
:102060001730019002920094081C00222AE00120FF
:1020700010700A6E1021002A00D00A21284A6846F2
:102080001730019002910094101C00211AE0009278
:1020900022481CE00092224819E00A6E1020002A13
:1020A00000D00A200A1C1C3206E00A6E1020002A0A
:1020B00000D00A200A1C0E3200946C46173402909D
:1020C0000194002001F063F81CE00092081C00213C
:1020D00004E00D1C1C35081C0092291C1A1C231C32
:1020E00001F0B0F80EE0081C02E00C4800E00C48DB
:1020F000191C221C01F0BFF804E0081C221C191C4A
:1021000001F0C4F86B46DA7D024B07B00120DA66B5
:1021100030BDC046B8040010540C0010C6040010B6
:10212000D404001010B506490B1C88331A68141C1F
:102130001E34A4006050013203210A401A6010BD11
:10214000B8040010054B0320191C88310A68013AB5
:1021500002400A601E329200D0587047B804001046
:10216000F8B5114D2C1C8C3420680130FFF726FE89
:102170000E4B0122D8629F6AAB6E061C02409A4247
:1021800010D1830703D420680230FFF7CBFFFF2371
:102190009B001E40B601BF10044B8C353743012213
:1021A0002F60DA600220F8BDB8040010540C001053
:1021B00030B50C4B0C489A6A031C8C331C68D30551
:1021C0009B0E910500D5403B856E921001210A407F
:1021D000AA4204D1E3188C300360024BD96001207D
:1021E00030BDC046540C0010B804001008B5084BB0
:1021F0005A1CD07F9A1CD27F000112021043DA7F52
:102200000333DB7F10431B031843FFF78BFF08BD2D
:10221000B804001038B5FFF795FF064903230F22D5
:10222000051C5C181540013325770011072BF7D1E9
:1022300038BDC046B804001008B5FFF783FF034B54
:1022400001228C331860024BDA6008BDB80400101C
:10225000540C001010B5064CA36E002B06D0FFF7EF
:1022600071FF044B8C3401222060DA6010BDC0463F
:10227000B8040010540C001010B5064CA36E002BCF
:1022800006D1FFF75FFF044B8C3401222060DA6037
:1022900010BDC046B8040010540C001008B5124B15
:1022A0001B68002B00D09847104B5A69002A15DD97
:1022B000012A07D1DA69002A04D09A610022DA6182
:1022C0000A225A615B690322191C91430A1E02D03B
:1022D000074A0121D166054A013B5361044B903303
:1022E0001A68024B5A6208BD78030010540C0010A3
:1022F000B804001000B5064B5A69002A07DD9A6938
:102300000F21044B1140D97712110133DA7700BD48
:10231000540C0010B8040010044B597F9A7F090137
:1023200012020A43197F0A435A677047B804001023
:1023300030B50B1C093B012B0FD8084A00239C1811
:10234000257FC45CA54205D0054B08395A68114366
:10235000596002E001330E2BF1D130BDB8040010FA
:10236000540C001008B50E4B1B68292B17D00829F8
:102370000DD0192913D1427808231A4202D0002225
:10238000027002E00F2303700723437005E000236F
:102390001A1CC25401330E2BFBD1FFF745FD08BDBB
:1023A000540C00101FB50D4B5C6F002802D00F229B
:1023B000944304435C676846211CFFF721FD68468F
:1023C000211CFFF7CFFF054A00236C46185D9918C2
:1023D000013308770E2BF8D11FBDC046B80400109A
:1023E0001FB5124B0F225C6F944304435C67104B84
:1023F0001B68292B01D0082C17D06846211CFFF739
:10240000FFFC6846211CFFF793FF084A0023991838
:10241000097F6846195401330E2BF8D1211CFFF7B0
:10242000A1FF6846211CFFF7FFFC1FBDB804001088
:10243000540C00101FB5114B114C1B68292B02D0F6
:10244000636F082B18D0616F6846FFF7D9FC616F86
:102450006846FFF76DFF0A4C00231A19127F694680
:102460005A5401330E2BF8D1616F6846FFF77AFF9B
:10247000616F6846FFF7D8FC1FBDC046540C0010C2
:10248000B804001010B50D4C631CD87FA31CDB7F73
:1024900000011B021843E37F1843E31CDB7F1B038F
:1024A0001843FFF78BFC0F23021C1A4022770211FE
:1024B000134000126377A07710BDC046B804001027
:1024C000044B5A6E16329200D258121A51424A41A7
:1024D000DA667047B804001000B5064B5A6E163223
:1024E0009200D1580139D150002901DA0D21D15083
:1024F00000BDC046B804001000B5064B5A6E163237
:102500009200D1580131D1500E2901D10021D15072
:1025100000BDC046B804001000B5094B5A6E163213
:102520009200D2580D2A03D11A1C2932127805E0E4
:102530009A18507F117F0001021C0A435A6500BDA2
:10254000B804001010B5084B0F245A6E16329200D2
:10255000D1585A6D58181440013104770D2902DC06
:102560005B1812111A7710BDB804001030B50F4B6C
:102570005A6E596D16329200D2580D2A07D11C1C82
:1025800029342478F02008402043586507E0981843
:10259000447F057F24012C435C650B114377034B7B
:1025A0009A180F231940117730BDC046B8040010A7
:1025B00008B504480022011C1C390D23FFF717FC45
:1025C00008BDC046F004001008B504480022011CF4
:1025D0001C310D23FFF70BFC08BDC046D4040010CE
:1025E00008B504480022011C1C310D2300F09CFD9D
:1025F00008BDC046D404001008B504480022011CE0
:102600000E390D23FFF7F3FB08BDC046E2040010AE
:1026100008B504480022011C0E310D23FFF7E7FB2B
:1026200008BDC046D404001008B504480022011CAF
:102630000E310D2300F078FD08BDC046D404001013
:102640000C4A0023111C46310B70111C47310B70D2
:10265000111C48310B70111C49310B70111C4A318F
:102660000B70111C4B310B70111C4C314D320B7027
:1026700013707047B804001000B5074A011C04230A
:1026800000208A1804E0D118463109784000084338
:10269000013BF8D200BDC046B804001030B5074A6F
:1026A00000238918012206E0CC18051C4634154089
:1026B000257040100133042BF6D130BDB804001052
:1026C00038B50020FFF7D8FF084C051C0021207FFB
:1026D000FFF7E4FF25770420FFF7CEFF0421051C58
:1026E000607FFFF7DBFF657738BDC046B804001098
:1026F00010B50020FFF7C0FF034C20770420FFF740
:10270000BBFF607710BDC046B804001010B5054C83
:102710000021207FFFF7C2FF607F0421FFF7BEFF8B
:1027200010BDC046B804001010B5094C231C8C33F2
:1027300018680130FFF742FB064B021CD8620F23DA
:102740001A4022770211134000126377A07710BD60
:10275000B8040010540C001010B5094C0021201CC6
:102760000D22FFF73DFB201C0E3000210D22FFF74C
:1027700037FB201C1C3000210D22FFF731FB10BD60
:10278000B804001010B50C4B00211A1C187F1C78DF
:1027900001312043187701330E29F7D1936E002BB6
:1027A00008D0064B1B690D2B04D1137F111C293156
:1027B0000B70537310BDC046B8040010540C0010C9
:1027C00010B50C4B00211A1C1C7F187801312040D9
:1027D000187701330E29F7D1936E002B08D0064BE2
:1027E0001B690D2B04D1137F111C29310B705373FE
:1027F00010BDC046B8040010540C00107FB5002373
:102800000C4A0D251C1C1118097F01306E46995584
:10281000C60F8542664176420133111C30400E2BB3
:10282000F1D100236C46185DCA18013310770E2BC6
:10283000F8D17FBDB804001010B5074B5A6E1632A0
:102840009200D1585C1801392077D150002901DA63
:102850000D21D15010BDC046B8040010034A00231A
:10286000111C943198320B6013607047B80400104B
:10287000034B012194331A684A401A607047C046DE
:10288000B8040010044A002313678C321360034B12
:102890000122DA607047C046B8040010540C0010E2
:1028A00008B59A4B0F20996A994A8B1018408911E4
:1028B000013852560E2800D9C1E000F0EBFF081194
:1028C0001A2327C02EC0C037C0C0C03B3F00002A1B
:1028D00000DAB4E08F4B9A18403200239371A9E0DC
:1028E000002A00DAABE08B4B01209A18403290713D
:1028F000A4E0002A00DAA2E0864B9A1840329279CE
:10290000DA6697E0081CFFF797FF93E0002A00DAE9
:1029100095E0101CFFF7D4FD8CE0002A00DA8EE071
:102920007C4B596E16318900CA5083E0081CFFF7B2
:1029300057FD7FE0081CFFF735FD7BE0002A00DA39
:102940007DE0101CFFF75AFF74E0724B01209833B2
:10295000186073E0FFF7E0FD6CE0FFF793FF69E0BC
:10296000FFF726FE66E0FFF7EDFD63E0694B00220E
:102970005A665FE0FFF728FE5CE0FFF7F7FD59E0DD
:10298000644B0120586659E0FFF72AFE52E0FFF73A
:10299000CBFE022052E0FFF72FFE4BE0FFF726FCB4
:1029A00048E0FFF735FE45E0FFF7D6FE42E0FFF7CF
:1029B00031FC3FE0FFF738FE3CE0FFF79BFC39E0DD
:1029C000544B00221A6635E0FFF7A6FC32E0514B6B
:1029D0000120186632E0FFF741FF2BE0FFF72AFDE8
:1029E00028E0FFF745FF25E0FFF74CFD22E0FFF769
:1029F0008DFE1FE0FFF72EFC1CE0FFF7C3FE19E081
:102A0000FFF776FE16E0FFF737FC13E0FFF7D8FE7E
:102A100010E0FFF715FE0DE0FFF740FC0AE0FFF7BE
:102A20005BFD07E0FFF74CFE04E0FFF765FD01E00A
:102A3000FFF702FC012001E00120404208BD982B75
:102A4000BED03EDC382B9BD01DDC1C2B00D187E791
:102A50000CDC0C2B00D178E702DC002BEAD0EBE792
:102A6000162B00D176E7182BE6D176E7282B00D17C
:102A70007CE702DC262BDFD175E72C2B00D179E730
:102A8000362BD9D179E7662B00D18AE70CDC4C2BA9
:102A900000D17CE702DC3C2BCED175E7562B00D170
:102AA00079E75C2BC8D179E76C2B00D17FE702DC9A
:102AB000682BC1D178E7762B00D17BE7882BBBD17F
:102AC0007BE7E62B00D19BE726DCC82B00D188E70B
:102AD0000CDCA82B00D17AE702DC9C2BACD173E78D
:102AE000B82B00D177E7BC2BA6D177E7D62B00D146
:102AF0007DE703DCCC2B00D09EE775E7D82B00D117
:102B000078E7DC2B00D097E777E7C046540C00103D
:102B1000645F0000B8040010F32B00D17CE70EDCEA
:102B2000EC2B00D172E703DCE82B00D084E76AE7E6
:102B3000F12B00D16DE7F22B00D07DE77AE7F62B81
:102B400000D16FE703DCF52B00D075E767E7F72BC3
:102B500000D16AE7F82B00D06EE769E738B5184C6A
:102B6000231C8C331868FFF729F9E26E154BA26617
:102B70000022E266DA6003229862251C10401C1CC9
:102B8000022809D090420AD0012802D0FFF788FE1F
:102B900007E0FFF7E5FA04E0FFF758F901E0FFF777
:102BA00007FB002807DDE368002B04D12B1C8C33C6
:102BB0001A6812181A6090352B681B182B6038BDE4
:102BC000B8040010540C0010034B0122DA660F22E7
:102BD0009A775A771A777047B804001010B5054CE9
:102BE0000549201C00F01AFFFFF7EEFF0123636682
:102BF00010BDC046B80400109C07000000B5074B8C
:102C000000201B680F2B08D1054B1A78824204D193
:102C10001868044B1840431E984100BD8400001002
:102C2000B804001000FFFF0038B5164B1A1C98328C
:102C30001268002A04D0144B1D6801231D4001E0D6
:102C400094331D68114CA3689D4202D16268002A2A
:102C500016D0002D02D1002B0AD111E00C4B1B68BD
:102C6000002B02D06168281C98470023636006E0AF
:102C7000074B1B68002B02D0281C291C9847A56015
:102C800038BDC046B804001098030010540C001062
:102C90009003001013B5002300930193244B1B688D
:102CA000002B02D0684601A998472249009B08786A
:102CB000214A00280CD0002B02D00223137035E0EB
:102CC0001378013BDBB21370002B2FD10B7009E09E
:102CD000002B0CD11378002B28D0013BDBB21370F2
:102CE000002B23D1154A1360154A13601EE01449C6
:102CF0000968581A44426041400010701148446904
:102D0000021C002C04D08B4202D10A2343610DE047
:102D100000290BD10A21516101999361D161084ABF
:102D20001360064B02221960034B1A7013BDC04694
:102D3000800300109C03001084030010880C001016
:102D4000840C0010540C001008B5FFF7A3FF08BD59
:102D500010B5094C20600948016009490A60094A18
:102D60001360094B029A1A60084B039A1A60084ACA
:102D7000084B1A6010BDC04690030010800300107D
:102D80008C030010880300107C03001084000010E6
:102D9000492D00007803001008B5084B084A19684F
:102DA00012688A1A1A6006D5FA2252001A60054B78
:102DB0001A6801321A60FFF737FF08BD880000105B
:102DC0007C03001098030010F7B50E1C0E21051CA3
:102DD000019200F023FE1A4B03240C279E420FDDC4
:102DE00009236B7301232B7328E0301C0A2100F0A8
:102DF00009FE301C29550A2100F0AEFD0134061CE5
:102E0000002E06D0E30F0022A7425341DBB29342CB
:102E1000EBD1019AA31A033B2B70621B2B1C01E020
:102E2000195D5973013BD1180229F9D10F231C1BDD
:102E3000002301E0013C2B55032CFBDCF7BDC04611
:102E4000FFC99A3B38B50C4B01221A700B4B02227A
:102E50001A700B4D0B4C08E01868884208D01B68AC
:102E60002360FFF799FFFFF715FF2B682168024ADF
:102E700010780028F0D138BD9C03001084030010A6
:102E80008803001094030010F7B51C4D9B235B00D2
:102E90000E1C1B4AE95C1B4BAC5CEB5C002902D0AE
:102EA0000F22144002E08021072449009A22520098
:102EB000AF5C154ACB1AAA5C3435BA1A80277F005A
:102EC000791A009107210C1B013210490194FEF779
:102ED000B0FE00230E4F33704124FF35301CFEF747
:102EE000F5FE2A786B783018D31A391C221C01346D
:102EF000FEF79FFE013D462CF0D1F7BDB80400104F
:102F0000370100002F01000035010000745F000050
:102F1000815F000070B5434B434C1A1C9432126819
:102F200090B0A061E161002A17D118280BD1C32904
:102F300009D13E4A12680F2A05D1181C38300E21DB
:102F4000162200F0DDF8A369182B04D1E369332BB6
:102F500001D100F07FF8FFF737FE0A23314D63619E
:102F6000334E01232B678C35FFF7F8FD2B68B342F6
:102F700016D006DC2F4A93420DD02F4A93423AD105
:102F80001DE02E4A934210D02D4A934220D02D4A64
:102F9000934230D10EE0254B1B680A2B2BD112E057
:102FA000224B1B680B2B26D10DE0204B1B680C2BF2
:102FB00021D108E01D4B1B680F2B1CD103E01B4BDC
:102FC0001B68102B17D1FFF72FFEFDF780F812E0DA
:102FD000164B1B680F2B0ED11B4C2368002B0AD0FD
:102FE000684608A9FFF750FF2368684608A9984774
:102FF0002B6827332B60154B1A68154B106819681E
:10300000884205D012681A60FFF7C6FEFFF742FE3D
:10301000044B1B6F002BA7D1FFF706FEFFF712FF33
:1030200010B070BDB8040010540C001084000010E3
:10303000130D0000070C00006A0C0000990D000041
:103040003E270000790D00008C030010880300105B
:103050009403001070B5254C23681D68FFF7F2FE3D
:1030600023681A689542FCD01E68FFF7ADFD204B1F
:103070000A22204C5A6118229A611522DA61231C17
:10308000903300221A60FFF79FFD2D36012323673E
:10309000FF36164C184D0AE0FFF760FD23682A68DA
:1030A0001968914203D01B682B60FFF775FE2368F7
:1030B0001B689E42F0D10F4C1820231C9033002136
:1030C0001D68FFF727FF0D4B281C196800F044FC12
:1030D0003834011C0422201CFFF776FE044B182212
:1030E0009A610022281CDA6170BDC0468803001076
:1030F000540C0010B8040010940300107C0300105E
:10310000F0B501240DE005780B1C254006E0C65CF7
:10311000ED0077083D43C554351C2540013BF6D5ED
:10312000013A002AEFDCF0BD30B504E0845C8D5C30
:1031300085548C5401329A42F8DD30BDF7B5099DB3
:103140000AAC2678089F2C7894461D1C002A0DD1C5
:1031500018E063465B5D4A5DD218131901920024A2
:10316000B34201DB9B1B012443550135BD42F0DD19
:103170000AE0CA5C12190024B24201DB921B01244E
:10318000C2540133BB42F4DD099B1C70F7BDF7B597
:10319000099E0AAC2778089D347800282FD0002992
:1031A0002AD01E1C9446002A0ED1013F18E0634627
:1031B0009B5D8A5DD21A131B00240192A34201DA9F
:1031C000DB19012483550136AE42F0DD37E0CA5CDD
:1031D000121B0024561C01D13A1C0124C254013395
:1031E000AB42F4DD2BE0D15C49420C1B211E01D027
:1031F000E1190124C1540133AB42F4DD1FE0002981
:103200001BD0181C002A06D10EE00E5C135C0130A6
:10321000F31A1C1BE40FA842F7DD10E0CA5C01336F
:10322000141B013462425441AB42F7DD07E0D15C2C
:10323000013349420C1B611E8C41AB42F7DD099AF8
:103240001470F7BD70B5049D01242C70141C002966
:1032500005D10BE0065D0A5D96420BD101349C421C
:10326000F8DD05E0815C002904D101329A42F9DDE4
:1032700000232B7070BD00B503E043185B78435406
:1032800001319142F9DB0023435400BD00B504E055
:103290008318013B1B788354013A8A42F8DC0023EF
:1032A000835400BDF0B5114B1A785B78825C1A40EC
:1032B00000D040220E4C0F49231C261C04C32C3680
:1032C00000221A6001240A1C123117785578C75D54
:1032D0003D4202D01F6827431F60023264008A42C9
:1032E000F3D10433B342EBD10020F0BD81010010D3
:1032F0001C0E0010CD00001030B512234B43334A92
:103300000131D3188A0051181A785C78825C144213
:1033100004D02F4A5F245218947054709A78DC7845
:10332000825C144204D02A4A7C245218533214700E
:103330001A795C79825C144204D0254A7C245218A4
:10334000A33214709A79DC79825C144207D0204C45
:103350005F226418251CA235A1342A7022701A7AC3
:103360005C7A825C144204D0194A7C245218A03240
:1033700014709A7ADC7A825C144204D0144A7C2459
:103380005218503214701A7B5C7B825C144207D056
:103390000F4C5F226418251C523551342A7022705C
:1033A0009A7BDC7B825C144204D0094A2E2452189A
:1033B000A43214701A7C5B7C825C134204D0044BF0
:1033C0005918F43127230B70002030BDCD000010B8
:1033D0008C0C0010F8B52D4C071C0025201C20215A
:1033E0004F22FEF753FC002D04D0221C7C233932DF
:1033F00023701370231C4F33002101351970503492
:10340000052DEBD1214B2D22181C38300270181CD1
:1034100037300270A1209A705A7040005F221A540F
:103420001B481A54A320400019541A4908784978B7
:10343000385C014204D0191C533152330A701A709F
:103440000024211C381C0134FFF756FF0A2CF8D148
:10345000114D124E00242B786A78FB5C1A4201D081
:10346000315905E03059FEF731FC0D49091A0A318E
:103470000C48043400F0DCFA0235242CEBD10A4964
:10348000084800F0D5FA0520F8BDC0468C0C0010A5
:1034900041010000810100108C000010A00000100C
:1034A00083010010CC0D0010895F0000F0B585B0DD
:1034B00001900027FDF784FA6A4C3E1C6A4A754267
:1034C000754113687D19012B05D168480D210C2227
:1034D000FDF714FB02E0002B00D1CDE0002303AA8E
:1034E000537023687F210B405C2B00D198E02ADCCD
:1034F000382B00D18EE013DC072B6AD006DC022BC0
:1035000000D193E0062B00D0B6E041E0212B00D1A2
:1035100084E0232B00D187E01C2B00D0ACE081E0BD
:103520004F2B4ED007DC3F2B62D0402B62D0392B83
:1035300000D0A1E064E0542B76D05B2B3FD0502B21
:1035400000D099E06AE0732B66D010DC662B3AD08D
:1035500005DC5E2B56D0622B00D08DE062E06F2B35
:103560003BD0712B52D06D2B00D085E02DE0792B14
:103570004AD006DC762B4BD0772B3DD0742B7BD1F9
:1035800046E07D2B23D07F2B25D07C2B74D135E0DA
:1035900031231370022E4BDD231C083B1B6819409E
:1035A000542908D0032E43D0231C0C3B1A687F23D8
:1035B0001340542B3CD14C2203AB1A7038E0322319
:1035C00035E0332333E0342331E035232FE0362355
:1035D0002DE037232BE0382329E039231370062E02
:1035E00026DD231F1B6819404723232920D11EE015
:1035F00030231CE02D231AE0412318E0422316E07B
:10360000432314E0442312E0452310E046230EE058
:1036100048230CE04C230AE0502308E0522306E044
:103620004F2304E0552302E04E2300E049231370AA
:10363000ADB203A8291C0022FDF7D6FA23681A06AA
:1036400005D5E91D89B20A480022FDF7CDFA2368A5
:10365000DA0572D50735A9B206480022FDF7C4FA8B
:103660006BE0C0461C0E0010900100101F3C0000D3
:10367000F4400000915F000023680122134206D04D
:10368000A818C0B2002107220223FDF717FA236809
:103690000222134205D0A81DC0B200210623FDF767
:1036A0000DFA236804210B4205D0A81DC0B20222E6
:1036B0000623FDF703FA236808210B4205D0681C96
:1036C000C0B207220223FDF7F9F92368DA0606D50E
:1036D000681CC0B2042102220623FDF7EFF923681B
:1036E0009A0606D5681CC0B2002102220623FDF707
:1036F000E5F923685A0606D5681CC0B204210722E2
:103700000223FDF7DBF923681A0607D5281C0930C8
:103710000222C0B20821131CFDF7D0F92368DA0594
:103720000BD5EDB2281C0930C0B20B210A35FDF7CC
:10373000AFF9E8B20A21FDF7ABF9013604340C37D2
:103740000B2E00D0BAE61B4803210622FDF7D6F95E
:10375000194D1A4E1A4F0024019A2B78D35C6A78BF
:103760001A4205D0A3009859395D0922FDF73CFAA9
:1037700001340235092CEFD1FFF740FA002814D0AC
:1037800006240321201C00F0E7F80321C5B2201C09
:1037900000F038F9281CC9B2FDF77AF9092C01D1DB
:1037A0000B24EEE701340E2CEBDDFDF713F905B029
:1037B000F0BDC0465C3B00008C000010940100107E
:1037C000C400001070B5041CFFF76CFD201CFFF74F
:1037D0006DFE0A4B1B78002B0ED0201CFFF7FAFD64
:1037E000074CC8235B00074EE518211C301C5034E1
:1037F000FEF714FAAC42F8D1002070BD9D03001012
:103800008C0C0010373B000000B589B000280ED0AA
:10381000FDF7A1F801A80921FEF7F2FA6846123077
:103820000A21FEF7EDFA01A8FFF7CCFF08E0FDF74B
:103830009AF8044B1B78002B02D00348FEF7EEF9F0
:1038400009B000BD9D030010935F000000B5FEE7C6
:1038500000B5FEE708B50A4B0A4A0B4903E01078A9
:103860000132187001338B42F9D3084B084900220A
:1038700001E01A7001338B42FBD3FCF73DFEFEE7FB
:1038800000000010EA5F0000B8010010B80100104D
:10389000480E001002B4714649084900095C49000D
:1038A0008E4402BC7047C04603B4714649084000CC
:1038B0004900095A49008E4403BC7047002934D09E
:1038C0000123002210B488422CD301242407A142F2
:1038D00004D2814202D209011B01F8E7E400A142AF
:1038E00004D2814202D249005B00F8E7884201D34A
:1038F000401A1A434C08A04202D3001B5C08224322
:103900008C08A04202D3001B9C082243CC08A04292
:1039100002D3001BDC082243002803D01B0901D07E
:103920000909E3E7101C10BC7047002801D00020F3
:10393000C04307B4024802A14018029003BDC0462C
:10394000D90000000029F0D003B5FFF7B9FF0EBC85
:103950004243891A1847C046002941D010B4041CBC
:103960004C40A44601230022002900D549420028EA
:1039700000D5404288422CD301242407A14204D21E
:10398000814202D209011B01F8E7E400A14204D2FE
:10399000814202D249005B00F8E7884201D3401A15
:1039A0001A434C08A04202D3001B5C0822438C0837
:1039B000A04202D3001B9C082243CC08A04202D3A1
:1039C000001BDC082243002803D01B0901D0090991
:1039D000E3E7101C6446002C00D5404210BC704741
:1039E000002806D003DB0020C043400801E080200F
:1039F000000607B4024802A14018029003BDC04669
:103A0000190000000029EBD003B5FFF7A7FF0EBC9B
:103A10004243891A1847C0467047C04600B500297E
:103A200005D000230139037001300029FAD100BD0F
:103A3000F8B5041CA30719D1231C04CB0F4D104E5D
:103A400050199043021C201C32420FD1181C0B4FFE
:103A500004CBD5199543354208D1181C074F04CB28
:103A6000D51995433542F1D000E001300378002BA1
:103A7000FBD1FEF734F9201CF8BDC046FFFEFEFE68
:103A8000808080802578000D0A413A200020202582
:103A9000633A20000D0A4D3A20002020473A2025A5
:103AA0003032780D0A0053455249414C20434F4E65
:103AB000534F4C450025732072656164790D0A00EF
:103AC000444D31314343000D0A4279652E2E2E0DAF
:103AD0000A004C43443A25303269202D20256900E4
:103AE0002573202573202025694D485A005638003B
:103AF000202025692E2530336956004241543A2052
:103B000025696D560D0A000D0A25303278202000F7
:103B100057616974696E6720666F722064617461B1
:103B20002E2E2E0D0A00426164206D6F64656C0DAF
:103B30000A00526561642025730D0A004F4B004650
:103B400041494C4544006F6E006F6666004C43442B
:103B50002064656275672025730D0A00000000006F
:103B60005C000C000C7C287C7C447C24104828548D
:103B700008000C00384400443800201008103810A9
:103B80008040001010100040002010083844380019
:103B90007C006454484454281C107C4C54243854F1
:103BA0002004740C28542808543800500080500019
:103BB000102844282828442810045408384C5C78DD
:103BC00014787C54283844447C44387C54447C1415
:103BD000043844347C107C007C0020403C7C106C19
:103BE0007C40407C087C7C047C7C447C7C140838D1
:103BF00044787C1468485424047C047C407C3C4019
:103C00003C7C207C6C106C1C601C64544C7C44001C
:103C1000081020447C00080408808080040800000C
:103C200007080400000000BF01BF010905000007EC
:103C3000000700070007130A00002000E400FC0052
:103C40003F00E700FC003F002700040F0800000CC5
:103C5000011E01FF03FF032201E201C2190D000052
:103C60000E001F0011019101FF007E00FC00FE010B
:103C700013011101F001E0140A0000EE00FF011130
:103C8000011101BF01EE00E0013001100105030048
:103C9000000F000F0A050000F800FE0307070104EB
:103CA0000B060000000001040707FE03F80F0800E0
:103CB0000000000A000E001F001F000E000A11097C
:103CC0000000100010001000FE00FE0010001000A8
:103CD00010080400000004800780030D0700001096
:103CE0000010001000100010001008040000000078
:103CF000800180010D07000C000FC003F0003C00A4
:103D00000F00030F080000FE00FF01010101010187
:103D100001FF01FE10080000000002010201FF0186
:103D2000FF0100010001100800008601C7016101C8
:103D3000210131011F010E010F08000082008301E3
:103D4000110111011101FF01EE11090000300038CD
:103D5000002C002600FF01FF012000200F080000BA
:103D600080009F011F0111011101F101E10F080005
:103D700000FC00FE010B0109010901F901F00F0827
:103D8000000001000100C101F1013D000F00030F1F
:103D9000080000EE00FF01110111011101FF01EE09
:103DA0000F0800001E003F0121012101A101FF00B9
:103DB0007E0804000000008C018C01080400000053
:103DC000048C078C0312090000200070005000D8FA
:103DD0000088008C0104010401110900004800481A
:103DE0000048004800480048004800481109000009
:103DF000040104018C018800D80050007000200DDF
:103E000007000002000300B101B9010F0006190DFF
:103E10000000F800FC010603FB06FD05050505058D
:103E2000FD05FF050601FC01F8120900008001F004
:103E3000017C004F004F007C00F00180010F080062
:103E400000FF01FF01110111011F01FE01E0110935
:103E500000007C00FE0083010101010101018301DA
:103E60008211090000FF01FF01010101010101832D
:103E700001FE007C10080000FF01FF01110111018B
:103E80001101110111010F080000FF01FF011100D4
:103E900011001100110001120900007C00FE0083D6
:103EA00001010121012101E301E20112090000FFEA
:103EB00001FF011000100010001000FF01FF010AB7
:103EC0000500000101FF01FF0101010B06000100D7
:103ED0000101010101FF01FF10080000FF01FF01C6
:103EE00038006C00C6008301010110080000FF01CA
:103EF000FF0100010001000100010001160B00009C
:103F0000FF01FF010F003C00F000F0003C000F003B
:103F1000FF01FF0112090000FF01FF010F001C005B
:103F20007000E001FF01FF01130A00007C00FE00A9
:103F300083010101010101018301FE007C0F0800E2
:103F400000FF01FF012100210021003F001E140A93
:103F500000007C00FE0083010101010101038307D1
:103F6000FE047C0412090000FF01FF012100210072
:103F70007100DF008E010001110900008E009F0119
:103F80001101110111011101F301E21109000001F8
:103F90000001000100FF01FF010100010001110902
:103FA00000007F00FF008001000100018001FF0090
:103FB0007F1109000007001F007800E001E0017890
:103FC000001F0007190D00000F007F00F001E00145
:103FD0007C001F001F007C00E001F0017F000F1239
:103FE0000900008301C7016C00380038006C00C76D
:103FF00001830111090000010007001E00F801F80B
:10400000011E00070001120900008101C1016101C8
:10401000310119010D010701030100070008000A21
:104020000100181110133831303378717073C8C122
:10403000C0C38881808384848782C5C4C7C27574E5
:10404000777235343732151417120207020802014D
:1040500000030109030402040205030500062024ED
:10406000282C383C4044484C4669726D7761726533
:104070002025735F56380D0A00252D313073202519
:10408000732573000D0A5479706520273C636F6DAA
:104090006D616E643E203F2720666F7220706172F2
:1040A000616D730D0A00557074696D652025757317
:1040B0000D0A003F0025730D0A0D0A00564F5941A5
:1040C000474552203E3E200025630048656C700045
:1040D0004E6F20706172616D73004B657920707254
:1040E000657373003C6B6579313E203C6B657932BA
:1040F0003E202E2E2E0044756D70206D656D6F7202
:1041000079006C004C6F6164206D656D6F72790091
:104110007400546F67676C6520646973706C6179B3
:10412000206F757470757420746F20636F6E736F79
:104130006C6500620052656164206261747465722E
:104140007920766F6C746167650000000080015013
:104150000080025000800350FC3F0150FC3F0250A1
:10416000FC3F0350E2A4615F2314411B51026B77B3
:1041700092C0597101E4C920093C174ADD6C0EA4B4
:10418000BFD6C07D2BFE334861E3589E78E4F91B0F
:104190000ABA7369E9666F1D14F71A4A50FC05F6EE
:1041A0009D3CE99F314EE0F4DE3AE7FF9122C414D2
:1041B0008DEF2FC14E48A52C01B54B9F3D570723CE
:1041C0004C5962B7277A7915168F233E7576813858
:1041D000E5083FBE6A3BBC1D9DF93FF81FEB2E2052
:1041E000047F23A2F5152996A75B2F4C1004AD6917
:1041F000AF7B410BFC438E62F4F3943BC5958FC9B2
:104200003464876219E96D55769DADAF66381688BE
:10421000C205613B12C8AF571522978F0B825B9F77
:10422000A59F6EA12DE2EDC185324538C7376EBD21
:10423000426DFCC143CE07BBEEDE11F7529919B3B4
:10424000ED70FF3F0488CD3C06A8CCFECAD5D954FA
:10425000A336B81379999C02480D3778CE3167B5EB
:104260000875B59BEB843150C2F66CC9F539973CA3
:10427000BB193B7A109F2CA40D5226BA41A4F90613
:104280002FD75B610C4EDD535490905AF49ACF4A6D
:1042900016C60B83DC71FD32DAC3689F94BA356DA4
:1042A0001E4FB4DBA51D76A7FCD06DB9F36EEB54A1
:1042B0004DFD1C8373ED76C5AEC46F48263AAA4FF8
:1042C000362C8EA9B0B9D59A1C211E8D878636EF63
:1042D000C37CAE9BEFB408BCEF68A01D10CFE91102
:1042E000111E7430902560900BDA9224E44C12B9C0
:1042F0008DA5F18E52BB29D89261F4FDB0662D9048
:10430000C222397DAB70CAB78FCF6F6E65E56E8202
:10431000C216FB5FCBBBC9772ABE459EC810636E31
:104320004751BF3C9BFC5CF9FE3DC47083EAA99FEA
:10433000431DC32C439CF8C5EA208675CC6D2685A9
:1043400027E04CF546438F15F5BB287575CB3F2804
:10435000C1C0CA3A9A8EF80C88208D7344FE09A316
:10436000EEA0071EA6BD625DFBE7C92A8C512FB4E3
:1043700038199E901B195213F7CB575B79CD5D4AC4
:1043800006FD27460B34D33236E94E0FF6F3AE77EF
:10439000DDA853F961C9B366D7BD3C2091AA5C2D55
:1043A0003268579F4F98E567F61D7D008C6D7CBB8A
:1043B0007FF2A2ED9E816FBE822BD2309C4DD754EE
:1043C0004830BF8E2503BEB70D83682234F7A93667
:1043D0004E818E036E8AF41D3DEDEDE71D20139C8A
:1043E0008187A02D317FEBA071F0D8D29A04BF3322
:1043F0003EA49D294CDDA5CB7DF60B2F7C9B51DF88
:10440000611E9072C416E7B1626F7250033002757C
:104410007BCAFEAD41CF288A8EF94F91B32626AED6
:10442000164A07BECD8FFF6722B1C1A2FC4E53765C
:10443000B41B308C24F579CB3A95470E73136D94E9
:10444000BFA58D3601C3D89715BECEFA16FEBDD1D5
:1044500085E405E98AA223115BBE11EB88C92B0B09
:10446000131DA3099449357663F503C2A789C632A3
:10447000B52055CFBBA19A23BBE36EEBC8D7FDE5B2
:104480008B787894524C9E7944610A6936E1AE7516
:1044900013221E6B88C7A0DE99EAA375A35DE2E133
:1044A000E5E1112780BCB39CE55575C3328E0FCA78
:1044B000F8B118224770514E474E5ECFFE0050A90A
:1044C0002F2E306D1E1DE7EA1018D7C760293F0454
:1044D0008967F3E5DCE9CB439FC306C5BD2B4445A3
:1044E000E0426E802A5F8FA25943121E239C5CDF3C
:1044F000EE196E662057FB7C466DC353CA3771AC0C
:104500006984D80F41228CDE002A1316447808856E
:10451000B16B3D373A81FD8E7F62B2580CB7C373E1
:10452000C19A090DC37F1E256D7C3F6D7478675A53
:1045300067925938557F09CBD8808D370C65900626
:104540009D88E0B642A8BA313BEAD7E7673567CE27
:1045500073306F1DC3CE8625691D42461719168A12
:10456000741371E03B956E22DB8114DBA13414D00F
:10457000EF75C16AAFF00E37FCDBD30E1ED8EE2A02
:10458000A074B0A23B106764E4BD16E4A3472713F0
:104590008D69C39F24C222A7782BF8492EF827E300
:1045A00010AE60F353FCC2786039B67E72259F5E10
:1045B0007F8700EF31A152393D30C45C72659BE3C7
:1045C000635EB0040485B4385C548A83BB934C2E7C
:1045D000435BBF1F6097FD823AEE252C5BE200F73C
:1045E000C5E4B0A7131B810F716D5C8451048FDC8F
:1045F0007B9405E8DF1E7DC3CCB864427EF19F72D8
:10460000139FF563C4462073C0478FEA50BEEAD1BA
:1046100052E7EFE63FED0B79671E975461BD33F625
:104620002CD194C379760129F6BBCE50EEB29B9380
:104630002E6970A2D7E377E885EA65304C93B3EE34
:1046400017EFB2E1437707A1A4738E2B31E585E61E
:10465000228EC732F755DAF50044C236C9EF548CC2
:10466000A5614F01198778EE69DA60816FDF5D61BE
:10467000493EE5710CF4706EC67EE469A4036B22BA
:10468000CD490E69780389B8A7EC2EC1E8FCBDC2FC
:104690003A92A2BBBADC1C1D5DEA68CB412D90B2F8
:1046A0004919B7B327C71162A1974F1E30B4FF6BEA
:1046B000D4FF5EBC5EEA8C543CFAC39086DA069A5C
:1046C000FAA4DD55D2DB1A8308A7C637B63F63E4E8
:1046D00040E187AFEC8242314EB85CB6217A5F3E52
:1046E0002C2C27B35A13B0C9283EF48CB5B7E991E6
:1046F000AE1C4CDA9C72E95CC185DEA48048248B38
:10470000B1EB42829681652E7EEDACFE5EBA1F6FE4
:1047100031AE36E7ECC060B3478FD76A47BEC043BF
:10472000D8B7AA2A745D5CD3F74B129638F25DC8ED
:10473000FD41EB3782FC6DAA9BEB2C30857BF6119B
:1047400014C2EE4E15FAABE96A5BC6217784842C5D
:10475000BAC7E9E11E744ADE02653A55DBE46A85B0
:10476000B1B7CF6D948DA5C622727774BF8B4A33D3
:104770003CD117ECEDC5F86127083FE8872D2A7C6E
:10478000991DA5E1D6E21B4D97B67AD5757736937C
:10479000FF0241875B798952FB936CBC455354CF30
:1047A00037B63246C0DDE2EC439EB8613C531E157D
:1047B000AC0159BBABF85AC865F824F7969C9462D3
:1047C000FAE040B96EF31336C73C211A80E1C78482
:1047D000ED99A7EE7CCDEB4FB17EA07C17DE224990
:1047E0006771A8A7A868B08311F557A9828061D125
:1047F000851EC7D6A81F4DF1242B63A527D4AB581F
:10480000A506166AE611500DA612B4A19B222D3002
:10481000BE28E957F09C287F67C9C01FFA7182D86B
:104820003DEABBE1A849A319F195BB869FC3B963D3
:10483000F051DB5821720A24A37DF1872BD9E9AC12
:10484000BB16E2977B573B2100017FD83814C2BECC
:10485000EE427B7AB33472BA2CCE5887FF8EB3F611
:10486000C7F97C14DC6C8461EAB5B642084F7C342D
:104870004203B455308593CD2709D086C308EFC4D1
:10488000A76B1D95089D7530776E5114C8C73B25E1
:10489000599E0292BA0C3F4029119D10DBE29C64A4
:1048A0009A4C343C9A67A9A975339276535BC044FD
:1048B0009C37F1E2203DA26D2783DEB3B5A47CEEE8
:1048C000A77FC9FF487954662D0DBBE8EA71606384
:1048D0005E83F1CB3395FE60714923A6445E53F9A4
:1048E0003FF7163A47096E55371C247814D97241A0
:1048F0002589F723E4125929250C7D243E4468FDBF
:10490000265EC11540DCF01119B53295805EE21FBC
:10491000F8D8877F1457A191664CF64B8B56A5EBC0
:1049200092C11FBEE7BC323361D3FDD6A23FE6562B
:1049300093202667311C552275D056D5B17590A0AD
:104940001E44E2C8A4B72A862FA7FEF86D9CC40EA9
:10495000939924EA06003AF2FE9A477DA71B30A7F6
:10496000DBEDC73911A7175BEA806D25D17AC29BB1
:104970009B7037D3B3A470068F5AF11D9D684C2EDF
:10498000A78801E4BD226BF718091B2336B9C66A54
:10499000C9282CCEA3B8FF02FDF8FDA10842BA58E1
:1049A000B84181C70EBBA5E8BC8AA26E0D5952EE74
:1049B00003746A8E2FDBBEBCFE4C4EED5F26B31C2B
:1049C000B28C31DCC1FE2D55A9F30FD6DABF527F70
:1049D000AC5C810E18EC757B356D11E1A14FB5898A
:1049E0003CB27C0449DDAD1D6ECD3DC6C41358D923
:1049F00063061F713291ACF0F21FC6C8932D147676
:104A0000E58166AD73F858ED26E8319F6F5A655F12
:104A100039AA19489290AE0C54E96EF49ADFBC00A2
:104A2000EEE0D16E50D4D143EECE3E2434C9EA87B5
:104A3000E13B763B80B8E0C508B0F119C576390E88
:104A40003925E05F96F88C3341A9FDBE842EFD30F8
:104A50006824EF5BA8ED3FBE205A91244078389F30
:104A600096DCE4B80B28FD8F882B0ECB80DF4A390B
:104A7000AB0CD90F2BBA4B224166FF65210BC5F554
:104A8000B5AFA42BAE5C991B25FFB79293652EDFC3
:104A9000B91DA68FA12AB99032EF09497FD8BFBFAF
:104AA000ECF5CE4D4A3A9ED763496EE3613CEEA8E1
:104AB000DAC9994D08EABE3D4F6DB06CEF9EF230F9
:104AC000EEADB05409FD2747CF66F482A6002F282B
:104AD0001A235B3038FB624A8CC1930FA8BFAA200F
:104AE0001399921924C2806DD4A2DCDCF5921D6565
:104AF00026FF1C4C9E0779E2A45C3F3E687616EBCD
:104B00004037B2EF18A96A0F8422672E51D1BA0834
:104B1000B2456AF1DE372A30C483E2EB69EC4C9A85
:104B2000803D23B8BDD8692FD63C82529A3932973E
:104B300058CFEBB8FFC04C6BD3F06824C9C12CC967
:104B40006DF674512B9F98193FD45C3BA43DA35341
:104B5000164366AF258BB0524B1599F8BC8530CC07
:104B6000E56F519EF2E70A3DA3E5841EA0C5AC6D3A
:104B70001705B95F3D57E24BA23E5997DCF02DCAAD
:104B80003D29BA74C2486B3E56BD714A06358E79CE
:104B90008481A3AA7042695E19E91FD5A98C49DEF8
:104BA0000F0CA5E705E055ADF466ACE230D0073751
:104BB000A076866AFC065E816EB87EECF48FDAD64B
:104BC000336F82A31A6AA3B5896CDE021B09D5C9AB
:104BD0005365D5CEDE79B4F49ECFC4F954F40C29D4
:104BE000761466F7DC10EC4CF7EF50F6807E0CB9CB
:104BF000667364E46DF9A90DB26EFD3E807FC5F465
:104C0000D1F0F992D75809DC600AF05DF9B0EAA852
:104C10004B6F585E5F3C4B3F8BAF39C5840E8E8225
:104C20006CACF1308C2B375447AC274975D124DB61
:104C3000822AFFB658C842FF8AF1B90F1A6F259829
:104C40002340FE91FB99738FB473830D6632892FD5
:104C500032798EC6D42EDCD4043D2F618D78B11408
:104C60008BE8A25EBFF583B3050A5411763B822719
:104C7000DBACD26EB2FFDF1F56709791F32EE64485
:104C80007A7897DDDDD9A0EC8E1A12BC8566CAE968
:104C90005CC13A8E4CFE0064C5314A0DD7FF874E89
:104CA000E9B32C5F2FEAF69C228AC8D4C077391A60
:104CB000C70204E07D620403CE2934E19478EFCF8B
:104CC00064FCC7BDC80C535AC0F639E22AF73D54FC
:104CD000F06B837412D6A3DE7838D95B690827534A
:104CE000B53D06EFDF7A1D2550AD324B3B1254899E
:104CF0000A4CC004DC2D793A130997ADF74DC37CFB
:104D0000BFB0560456A5DB188373EAB9367FF02B83
:104D1000244345842BE4644C55B8882DC8F24B4895
:104D20004E25B9F0BD0F07F6C673384EC735D48986
:104D3000A29172E38223DEF209DC1CC19F5CEF3694
:104D400058D8055B3159E94852321383F801AFB79F
:104D5000414B549660755934AAAF1E1D825EF38E86
:104D60009FCB5ABC5640EB02A6E3CCC71BDDDC9CB4
:104D7000A016B49B1D1F9BBE21235410F8FC8EF877
:104D80004C683BA86151B8932165130BE0DF398370
:104D9000152C207F76B5B724262C096330EB96229C
:104DA0003B052DB99511563051756605DDDB840C38
:104DB000F549DF7E3CDFB217BE2D316FB0F0D2DE99
:104DC000B739DBA53A5E14A5A700E0718223BEEBDC
:104DD00065ADF6828D690176725EA4E050B59F3BA9
:104DE000BDF7AE1B4717D5FBCD0A8441E247F0F172
:104DF00012CD576F87772E9CF0AB0BC96DE26846DA
:104E0000C7F65D308E104FC7D020CA368C03BD392F
:104E1000244C265DF80CEB5D4AB8A16992F3B733D8
:104E200030A2597A37C392B86DE416B802DF4A91BE
:104E300089D832DE4FB1CA15F8883120C4CB7CDF67
:104E400059A5C5BFC765784AEA65F2C13587FE4FE7
:104E5000010B7D5CC86EA28DAC928FEEB83FF60F51
:104E6000439BBAB8C20B7C66867CDF245F4E25F27A
:104E7000406F02E55A97C474FEACCD95AFFC0FFDB0
:104E80001025A722ABB739F862AE781F0257C58943
:104E900054E5EDA5BE28C18CC490904D982E95BDCB
:104EA0002E9ABAED3582A4F653D4092A60A5FB2BBD
:104EB000B3F5DBC0A0F9E9AC3179DEBAC612887A65
:104EC00040269975A33879340A00F36FC7FD43DF94
:104ED0002FBB701D624FE24C0472526CD594940645
:104EE000763A7D7B14E177A6798403F21913FE24C8
:104EF000F1521B8FC98BC955D55EA6E3AA6DDB168F
:104F0000E5E78A8C9F62161958E33EDA1DB1748E6C
:104F1000D2242D40C1FEB6B5CEBAD5BB5578E160DE
:104F2000E957C5705210AA17268318C07D44C524BE
:104F30005AC837C4C20F2D83BABB328A10CC400680
:104F4000767F20B988C8CC4F7436C112DAC7627F29
:104F500048CD7E9F5B3F7654A42550F63374598725
:104F60002A44FB63C6E5B51D0C2A4055AAA2F8AF3A
:104F7000D163C2B9593964D61D19CC734D8AFC5F0F
:104F8000564EE3B6FCBDAA6941312B73BCFE1983B2
:104F900082D5C67ABD88A59D7372007C85C456FBF8
:104FA000F9C954E78795CEEA6A31152A7970E79FE7
:104FB000426ABABD9A977213C69CC183C13885DA1A
:104FC0006142C57E7E10157593966E77F8800779DD
:104FD00077A29AB2F9D405577B52FA743F5F8924BD
:104FE000AA9AD676631AB8DB5619E09127B67F26BF
:104FF000AB5F28C3BED2FD5B969FD12929D0D5EDEA
:10500000BA4CEB0E2E117DF97C19471B25DB820271
:1050100092F3363494F775D5C577069884DD60062B
:10502000F96EB0CDBD860388723617AB24BAF96C21
:105030002F47C49EC787F7711313C6DE3A5BF1187A
:1050400066DCC02C5B773E4FCDF6EF04FBA2867A80
:105050007A4CF392A2F392C218B509EACA795CE8D5
:105060005F34115DEF53ED4048693C42669D70B678
:10507000676D66FE0B729C2905F8D3E7F26A144A45
:10508000DC502DCAC3C508A4DDA3CBFE85D7E6F648
:1050900099C762E1108B2DE8EE9B52AB803D9D8459
:1050A0003A42A946376B84DD2054CF7A13F695082F
:1050B0008DAD64908FEF3A38FE0F20ECB248DA984D
:1050C000B55F0FDE551964CAD843A59FF285E33555
:1050D0008CCF28E3C88590788026AE0B686F03F4E8
:1050E000F20DB29F95936F703067050063EB240259
:1050F000C6C0DEA66EBD05EA4314D93F39B077A21B
:10510000EE7DC6C026A095C5A7E7522E9423210E9A
:1051100085CC5655CFC9B9B0B71C4F69E0825E78CF
:10512000F6B21DAA25DA869572F263488CF8B72785
:105130008376BC46D217E7D05C172574960467FACD
:105140001E682E0B1240DA93F5D9A58E85ECFC452E
:10515000F5A4483D1782D21F6195E7A4EAD71B4307
:1051600052B10CA48A83EF09982168925D1AB0A409
:10517000DCABD04C08DF7D34957BA3E3C1D180BA92
:105180003DE4D6CAE11290175D8031DF9B86342161
:105190005B6643164BA2D2141581C6154B14943E80
:1051A00049255E48A8CB30DD82140EC0B3F54EB45D
:1051B000D449F1537CE8388DC0ADE5CA97338B2ACA
:1051C000B7FBD49EAC1624C14315F6DA03D999D7A0
:1051D0001749F16EC0D9057DC84853F89A3D4DAFC7
:1051E0004D1B7B1DC8559D3CEA2A632D29C291B8F1
:1051F0008DC0A699B3DE32BD49353D7354BF46B963
:105200009BA6300CD202BDAC02A19D020BBCA974BE
:10521000479EE3B50A43F320F6468D8EF0463316DB
:10522000F7DCFC778BCF6D37E64C1EB91C2AD28891
:10523000DCE336DC7086642C5172B5F4E332434310
:10524000CCDE5C2AC7642F0C1D1F2B544A39A2C325
:10525000CA1F9C0CB1654F1020F80D1F4E7C817643
:1052600066DA99CBC306377FC03803E4238FF25F39
:105270008A2EFCF1F72A1AE2DB650E2A77860BAC40
:10528000623CBAFF484F6CDC29256769B1C25BD923
:105290006092AFE28A5BB1C62C646C8B41530C6F99
:1052A00040B6D68B69AA4A17C8B15CFF0B3E34B42E
:1052B00081D6063D36559A87F1D22949B16EC1DDB6
:1052C0000A71681A6179864D4D884E237ADCC9458A
:1052D000C8CF0CA2632212232906F778446CA1D010
:1052E00062C348D43BF33D2F2E296BDD34CBF99BB1
:1052F0002DE7947C17F456FF25A92494F4B379285C
:10530000F7CAC07EEC84771CB31FFCDCD5B489C41B
:10531000414C274D5B24454855134FAFC29674C886
:10532000789453B913F0DA06429B94BF6AA84F15DC
:1053300040CC209EA70F2B3D068A70DD3CCC8743D6
:10534000CD9220B4D5D87676A24E677D210483CB4A
:10535000B46C8E48C5FF378182B6A12EBC251BAF29
:105360000D5B1B21AA2A75BEEA3CD92B8AEEA5F952
:1053700070642A0F40034928C9CA2636615BF94385
:1053800089D50C92F99185D2D1452CC495341F0949
:10539000FA56EA01A0C5C9208DC46C180FFBCFB71F
:1053A00024AE8F901FBD5F886B3B1A71A42A310A0F
:1053B0004E65D54B3EEE321C40963977CC602720A7
:1053C0007052E48FDF8B9A4D07D75C2B5821C71D95
:1053D000BD202FE668E5350AE0530D653475506D44
:1053E0008CEF2F594250E150516875C93498636A67
:1053F00049E6CD5D3FBC1C5F092B454C60299724D5
:1054000055B81B6D45BB62F4B30C8A0DF25A11F707
:10541000B97E960A3C45EC9F70EDBA7ACE1AF4BF7D
:10542000B3D438127D1E35FD64CFD48394397718F8
:10543000F8744EC7FE7DE40C98A35866D93EDC9202
:105440007C616C0E532FA8B9C266385B9A20FB5B57
:105450006F104EFCF9A8574CD3BB7D6892AD0F7A04
:10546000A3ABC34E0E25621A4C7262F4ED1102B862
:10547000CA3D45C278B4F9548A72839768DCA24C5D
:105480005B2202E2E42E1EACC23A29658BC410DB1B
:10549000D5844EB8D0C1E77AEB014365D9FF35EA30
:1054A000214F4167F06280C41BA96453806955880D
:1054B00046266A1FE8C5B4903BED6519CEEA8DDD3E
:1054C0000DEBEE299CA6F0EE50CD7E72EF6EA0E9BA
:1054D000E31420E4580B2CAC4B4A48CC6A462FE628
:1054E0002EBC5943FC462C4BEAB564B8158C556567
:1054F000C42975D1B8CE2B6940E29B3E9EDA534752
:105500000F8012ED1BA6189E6DA4F5B6DDFCBEB390
:105510005DCE1D59D86B972E30C5E259CCEF798DF1
:1055200004829598185C1BE4FD7973DF0152D32542
:105530006DB0CC5F676966F08A536B10FE88FCEC37
:105540000E00B37BBF5B8E45C43AA16AE54E0A22CA
:1055500084218C43F024ECF0C860947B50F98DB426
:10556000C9D60272A2F4AEC5F850BAC1A9C927AD16
:10557000313031B4B6D50FEF442AB5A6DAE891A29E
:105580000865B79A04589ACE2A0B1DABAFE5FFE623
:105590000984E3B37E000ACAB58A521FA85620D6F2
:1055A000A4725DC05A67470C99431EDB511704066D
:1055B0006964ED143ED24FD08EC277DF15921693F8
:1055C0001A2E709E2BAAC8FE686EBBB41DD3BD7682
:1055D0006F0660782A7118B42100E38D3E4953CAE2
:1055E0004FD8DAEB5F30C3EBF1405B82F2AD5F770F
:1055F000246FD825A6E1E1C8B26F0D4E13CAB1776A
:105600002DC33E2DF9D9635168C3E482105BB650B7
:10561000FADAD1734B6BFC883D9E8C738E03243178
:1056200070E0E829D6A9E51005DC0FA445157E6ECB
:10563000DA09B4E70EB5DF725B0DF041F643CE2711
:10564000A22900E9BF05D93F9A2ED5F66F805AE40A
:10565000B12C7E4BA37A0AF728DD7783F3BC2E406A
:10566000EA7D0789377942FBF798ECE3A47444BBE1
:1056700019700855FC21CC1BB98D0C40A02B1722AA
:105680003E84F58F961256002CD2E094A605EFD2F8
:10569000FF71982206A82DF2901DA5E6823431D420
:1056A0007A0B225B37E7B419292B1BCF7AE8C55256
:1056B0007841DD94213C19046945CB03B598691400
:1056C000F608AFB8010525F4614B717C7C73542555
:1056D000978D07F2E2EADDADDE61107900634AE7FB
:1056E0009DDC7F6C1AF69A4CEA6C36F393E8EBFF7C
:1056F0006151A811F5409945C0CCBF317A586592E7
:1057000017551C89A04C1299CAB59025CDF9A61041
:10571000DB765D69A61A0E531E8BD06684EA0FA055
:10572000CBAA5A5CEFB4C7BB2537F6AF5B648BD20C
:10573000EF0D7A30B64A924141F393AEB3D0B09CAC
:105740003213B4C83363533615AEDA9CC58341C7F0
:105750007D7822D69CFE3137494CF9E09605504AB7
:105760006AA4329CADFEBB8D0EA384AFF0B78760F8
:10577000794E08DAE4C5E2A96FC9DB17F412078C89
:1057800062AA7BC3AD080BD22FB7412B2DE8BED741
:10579000D5FFDDE5EBF5DED03D8AC1E3DAE257E681
:1057A000B2FC7DE54186B11F2FF83E18EBA871E4ED
:1057B000DB433D38DC427B9DBCCE9D8A8170EDEEA3
:1057C000CDFDDCF0EF734E80DFD6B9F98C242E7955
:1057D000DF230A78E51D4E0B35F9C161C7817C587E
:1057E00021585BAFE3D2DBE0766AF6D089A2D632ED
:1057F000FD8F3DE92BE4D8ED48A865F7D339E6B92C
:10580000BB58D0B3312C143178ACB56D5CC774CEB5
:10581000BAEBC19975C0FBC78BD68B5D167F2E196D
:105820009E31C4A89CE03A36A44FE693B9EABC1F67
:105830000DCE10AE3A3F65BBDD13F21926A09CC613
:105840005515FCBA9FD295461CB2F382074CEC0D5D
:10585000C6736C394696E3395C006F5B1B5624C7F0
:10586000F2B94DC8481791D3C584764CD1C28B6626
:10587000DD90ED505657530D789AF6DF1B26E34F17
:10588000E651E8527103D8DC1928F517FEFE3CBD3D
:1058900053CD26D3C6F82DAC5A2894870A681E2605
:1058A000D59312F699173FCD498FDB2E5468E6E267
:1058B0005DD0393DB62CB2845BBBD7B6A1E5E29290
:1058C00055FB57DABF7A4F076726C12C352AF0F10E
:1058D0001B093268BA729805F926CF6EB88E1194FA
:1058E0006852112EDF9745905B017F5C45A3F7D08E
:1058F000903A3617D485528F8C0ECFE171017EE538
:105900002C176B866790977BA58E801BE86A196DB4
:10591000A68F53CA99EB442B0F0911F47058C20596
:1059200087BFCE1B925621A44B2DB694616DB16AF0
:105930003A80E4441961BD57A4F573B22129367247
:105940006807B5ED0FF7F838F0E006B9ADD71614D3
:10595000E5C3B36F7260CDF29AE023C81CB89240E1
:1059600043B72F6EE6A392C0775EB6D19EDA627916
:105970001BAD1956A6EF147A0643D706D7C53CD0FF
:10598000034A4A372CB5B92BB046C39E57E654FD9F
:10599000AEE607AFEFF0A234E7935FB3CFBB7B6F08
:1059A00078D45ABA8487AC952F114B03ACDFD8ABAF
:1059B000B33FA2A6D262E819768E4E79DE6E2D41F3
:1059C000A0045E9FDE6CB8A95B3A8812AC8D71E7CB
:1059D000F82648876DF666B0993C9CFE69C714614D
:1059E0004DDECE2100744A1AF04AD31C94368794B7
:1059F00099AB41740F15BCD282425169A9C697E890
:105A00000ACA69245D9AF89E557ADBFFAA0DAE6634
:105A10009A4D8520F2108D63CFB27FE37303C54B9F
:105A200050B076156056F927EA103D28103DC31B8B
:105A3000E779D7B0E3419BF92F70FF006A54160253
:105A40007A228AD19DC9DDC6128347A853816C167C
:105A50002A31CD5FB450813FBC7723DC1F0572A98A
:105A6000B5F3050FD90756D81B30002BE9FEE289A4
:105A7000071E45B0BAA328D2C4C4AC2268339E1A0C
:105A8000033B814DB83D2CD9415E460C467A868A4F
:105A9000BC056BD26324E09FB904FD0F3B27006473
:105AA00054C1BEBB2423328F33864E44DF1DCDB795
:105AB0001B434F79C47C2C128B36BE6DBD89B56FEC
:105AC000838E1C23D01E7BD788D9DEE39BB24F9EEA
:105AD000E5CD1E190CC49CC5447DD34F4F110394D2
:105AE000AFC28253E2BBA40AE36B923658C642FDB2
:105AF000CEA0545B975F58ECBA223ACDE950D2362B
:105B0000BC8CC5C85847D9923F07608148630E4E88
:105B100095EF275E1DCC6E8239A180BDAEAC5A7167
:105B20005A58CC8B7784BD16F60244213AD19C4456
:105B3000721697AE84B907B9DDE5D63700EFB5D454
:105B4000D62B7150206225E0F41655BDF53FDECC12
:105B5000D5169F49B02B48771871BFFC4B0F74CFF7
:105B60008857ADEFD4424E231DA3E435669D50BE49
:105B7000846F99C75EE8BD5C04453D16A50768358E
:105B800096B60A04DB4E8B67117A81598F5A3B3CDB
:105B900077BCD35840243D9B16B13BA0A67DE8FAC4
:105BA0003D60014FE3551C329F8E616C325526C417
:105BB00093127093B6D3DEDA93A52DF82AC9B4D622
:105BC0007059DD111CCBD6CDC070AB5E7C51E31A91
:105BD000B74A5BABC2860D674639207C8AA1132485
:105BE00054B451BC29C31999E5315C3702D1120173
:105BF000DE702DF52041E1D827761153B1457D4F58
:105C0000C1101BCB3A7CA7BCB8CB5B519B9B3347E5
:105C1000393FCAEEED8E2D311F07528EB8EA978BB1
:105C2000834C3496DB240CD721AB50FB5091B01938
:105C3000F38E140219414FD8CA88DBB79640A1AC45
:105C400042971282111CEE340E1E68D73086F2780D
:105C5000AFB753F5DC16483E7B868BA283D75C0931
:105C6000381D8F7D0318E68B047A262D4407DA4A07
:105C7000CF2729BEAC2793B9BE3F65A0C0EAC37742
:105C80002EEB9FAA383C1DFA73ED45C20B06551D3D
:105C90009CB4428639CDF484868447F6F688505900
:105CA00076118571B64FE8CFD66C7B58B9410D118E
:105CB0006074358AE2B37AF1205E9BC0D41F59A884
:105CC00089C6033A853EC8C6CFAC1ADE7E7720ADC2
:105CD00089D9273E36353B140936AE6BAFD337989A
:105CE000D7D388EF5FB315CB6E06C0F1B502014480
:105CF000A802BF1F94703D34BDDB39365E3EE90516
:105D0000E92F5FCBED3517A46388A532A176DB6060
:105D100001DB216A1162DF92911D1D914C22374EE9
:105D2000B32AA0AB97CF2FA1B54F2AD1DC110A40DF
:105D3000EED4CAE6187555886E74830587E7BAEC09
:105D4000A0BA2466B0812D9004683E08BB4D32C9CC
:105D50006EDAB718C02F44DFD7A5E96B6F863D1DFB
:105D60009C90D514F3A0D5AD50F50063475FB9B151
:105D7000F3C386E9474EE9C08C19B784C2EC8AA305
:105D80003407857C3FCE75961E61F376372858F42C
:105D90002B6ED7D201A5FDBF76A9625521E2DB9714
:105DA000BEF764E75FB9334EB846CB924D7944BC39
:105DB000DB86A39D19C93E7721A963E5BF38CB26B1
:105DC000D5F55F02F4485FD63C8CD9EA59E65F030B
:105DD000D54833E1680937112697A87337EC8A78DC
:105DE000B6BDD4B5C517FC30CF87E63A1B172DD703
:105DF000950D6771833AAF3EE324BC72162A137780
:105E00009B33505FA843B2C032D49D14AE90D61ECF
:105E10006150714F429D65F6655A56A6EB6633BBDD
:105E2000348F4177CD7D6329AE3D0E35B94964EE9F
:105E3000ED2501E64EC30EC5BC526BDBC323BB820E
:105E40004B9DE94901793C68DD72BFEA898FFB2DE2
:105E50004CEDD489C26A28A8E303E03D7EEB6A4D8D
:105E60004718E434F9937ADB88B44444E77A038032
:105E700015914D9283D4B3BF4BB8138F51954F0EEC
:105E8000B302AFF1336AB581A5B9B1D270BBB25BD1
:105E9000B94D16BE236A7F107CF3F69EE939458A18
:105EA000F68220685EC2D709CAA34C53AF846EFD48
:105EB0002AAA8D0D9EA461E3CE107DF2DAE50E33A1
:105EC0005512A8849093B0FE1600DADDE6400A8CE5
:105ED00094D77B09B5D8D1EB8EEC9F04E3A19BBA94
:105EE0003B29ED9D6D265B14EBC5A53372BD6800A3
:105EF000A280F63E3A14A0297B518656A88CB19B0D
:105F000039E2A8F309040AA02AACB85242DD164DC2
:105F100002CAA43D66DD3B523A40D5D43C5328F931
:105F20003E7A351CEC7B7C68FDE24CB8ED99E9DBF0
:105F3000917EFBC830EE99D1C0E25DEDE2CF212E1B
:105F400092E6D3321D39CE67A838494E7C55DA9493
:105F500074EB885565D3175817833EA122705427D8
:105F6000D25045B80304050A08060BFF0209070DC5
:105F7000010C00FF2025692025692025692D256950
:105F800000202025633A256900202020205F5F7CC7
:105F9000002C0044697370206F66660D0A0055532B
:105FA00045520046004700424547494E0052414491
:105FB00000442E4D59005052474D00555345522034
:105FC0002020006620200067202000424547494EDF
:105FD00020202020200052414420202000442E4D2B
:105FE0005920202000432020200005000000FFFF52
:105FF000FFFF4D000000B3400000000000003D1016
:106000000000CB400000D0400000CE400000FF0068
:10601000000001080000DA400000E4400000824077
:1060200000000000000021060000F6400000D04003
:1060300000000241000000000000C1060000044111
:106040000000D0400000104100000000000059088E
:10605000000012410000D040000033410000000069
:106060000000E905000035410000D04000000F00AD
:106070000000F40100000401030102010104110405
:106080000F041704160118010000BB5F0000C35F76
:106090000000C75F0000CB5F0000A55F0000D65F77
:1060A0000000DD5F0000E55F0000B65F0000001744
:1060B0001B243E425369750502050804080B0804B9
:1060C000040501050409080904060807020602047C
:1060D00002060106040701030803040C080D020C64
:1060E0000203020C010C040D010D080D0408020846
:1060F0000807080202070408010804090209010A46
:10610000080B020A0201080A010A040B0102080234
:1061100004100811021002110810011004110112DC
:106120000212011302130812080F081204130113BC
:106130000414021401150215081408170814041594
:106140000115041702170119081A0219021602197B
:106150000119041A01160816041B021B081A081854
:10616000021A041B011B04180818040B0420202029
:1061700020202020202020000000010000009E5F41
:106180000000A35F0000A55F0000A75F0000A55FFF
:106190000000AD5F0000B15F0000C53A0000B65FCF
:0261A0000000FD
:00000001FF
